:040000002500FF0ACE
:0200FE00FB0CF9
:10010000060000000000FF0C06004606850A7F0A74
:0201FE00C40C2F
:100200002600D90C020083067F0AFF0C2700280075
:1002100069000400FB0C4701060000000000070213
:100220000600FF0CFF0C020C2A00FE0CEA02160B63
:1002300046073E0BFF0CFF0C020C2A00DF0CEA0203
:100240001F0B46073E0BFF0CFF0C050C2A00FC0C95
:10025000EA02280B46073E0BFF0CFF0C0A0C2A0093
:10026000FD0CEA02310B46073E0BFF0CFF0C4A0C5B
:100270002A00EF0CEA023A0B4606FF0CA801280000
:1002800043074B0B290243074D0B06002700FF0FC6
:0E02900043060300090B3F0C2900E900090B8F
:080400000F000F000F000F00B8
:021FFE00EE0FE4
:00000001FF
